:10000000F83066000828061A0828861A11280328DE
:100010000530A0000730A1000830A2000030A30086
:100020001A280530A0000730A1000030A2000130DE
:10003000A3001A280610861006150310200C0610BF
:1000400003180614000000000000210786140310A6
:10005000A10DA10D8610A107210C000006100318A8
:10006000061422070310A20DA20DA20D861422076A
:100070000310A20D861022070310A200A20C061086
:10008000031806147D302318A20700008614000010
:100090000000000086100830A400A20C86100000AA
:1000A0000000061003180614000000008614A40BBC
:1000B0004D28841286100000000006140000000085
:1000C00086140000000086100000000006100000EA
:1000D00000008614000000008610000000000000F0
:1000E00000000610000000008614000000008610CA
:1000F000000000000000000006140000000086144C
:100100000000000086100000000000000000061043
:1001100000000000861400000000861000000000AF
:0A01200006100611061486140728C5
:00000001FF
